:0200000480007A
:100000006F00C004732F2034930F8000630AFF0336
:10001000930F90006306FF03930FB0006302FF038A
:10002000170F0080130F0FFE63040F0067000F000F
:10003000732F203463540F006F004000136E9E53E3
:10004000171F00002320CFFD6FF09FFF732540F1A5
:100050006310050073251030635805000F00F00F82
:10006000130E100073000000130E00009702000032
:10007000938282F973905230735020307350303035
:1000800073504030970200809382C2F7638C020065
:10009000739052109302B01A739022307323203061
:1000A000E39E62F873500030970200009382420191
:1000B00073901234732540F173002030130E20002A
:1000C000930200001703000013030301E70203007B
:1000D0006F00000C170300001303C3FF639A620A4A
:1000E000130E400013020000170300001303030166
:1000F000E7090300631EC0091302120093022000E7
:10010000E31452FE130E5000130200001703000008
:100110001303430113000000E7090300631AC0073B
:100120001302120093022000E31252FE130E60002D
:1001300013020000170300001303830113000000E3
:1001400013000000E70903006314C0051302120046
:1001500093022000E31052FE9302100017030000E8
:100160001303C3016700C3FF93821200938212003E
:1001700093821200938212009382120093821200E3
:10018000930E4000130E70006394D201631CC001F3
:100190000F00F00F63000E00131E1E00136E1E00F2
:1001A000730000000F00F00F130E1000730000002A
:1001B000731000C0000000000000000000000000FC
:0401C000000000003B
:1010000000000000000000000000000000000000E0
:1010100000000000000000000000000000000000D0
:1010200000000000000000000000000000000000C0
:1010300000000000000000000000000000000000B0
:081040000000000000000000A8
:040000058000200057
:00000001FF
